:020000040000FA
:040000000000B8281C
:040004000034003490
:06000A00F000030E83016B
:10001000F2000A08F1008A018C1C46288C10051E8B
:100020001B28551C232850088500510886005208BB
:100030008700D5012328FF30850086008700013026
:10004000D500FF3041285308031D2C2800308500BF
:1000500086008700FF3041285309031D3128FF30F7
:100060004128D409541C3C285008850051088600BA
:100070005208870053084128003085008600870019
:1000800053098316920083129101B1288B131A0829
:10009000BC008C123B18A228BA1B752830088400BB
:1000A0003108840700083C02031D6028B10A0530AE
:1000B0003102031D6128B101B901FF30BA00B12836
:1000C000B101380884003908840700083C02031D88
:1000D0007328B90A05303902031DB128B101B901ED
:1000E000FF30BA00B128B901B1283C08BA00FF308E
:1000F000BB0000308A003A080F398C20CD004D0833
:1001000003198A28BD01CE01CD1FB128CD132808BF
:10011000CE00B128D617B128D70000308A00570882
:100120000F39820700340234823401340034003441
:100130000034003400340534013400340034003419
:1001400000340034CE080319A728CE03B128400894
:1001500084003D0884073C088000BD0ACD0BB1280F
:10016000D61771088A00720E8300F00E700E090017
:100170004130C000BD01C101C201C301C401C501BC
:10018000C601C701C8012030B8008312B901380880
:1001900084003908840783168D000C140C08831220
:1001A0008000B90A15303902031DC7284C30B2004F
:1001B0004930B3005430B4004530B5003030B6009B
:1001C0003230B000B1012930B800BA01BB01BD0125
:1001D000D6010130D3009F01831607309C00063002
:1001E0009F0000308600F0308500F03087008312D9
:1001F0008316FF30920083127F30920083162030E6
:100200009900043098008312903098008B170B17D8
:1002100083168C148C168312D61B0F290C29D60139
:10022000BD01BB0101308A003A080F391A3E03189C
:100230008A0A8200B8282C292C2936292A292A2919
:100240002A292A292A2944293A292A292A292A29EC
:100250002A292A29BA010C294108D10042080F395C
:10026000D200420E0F39D000BA010C294108D30048
:10027000BA010C294108A8000830D8002830D9005C
:100280000130BE00BA0155294108A9004208AA0060
:100290004308AB004408AC004508AD000930D80065
:1002A0002930D9000530BE00BA0159088400000881
:1002B00083168C008312580883168D008C110C1540
:1002C00055308D00AA308D008C140C1183120C1E39
:1002D00067290C12D80AD90ABE0B5529B901BA01EF
:0402E000BB010C2929
:02400E00323F3F
:1042000000000000000000000000000000000000AE
:10421000000042004C004B00300030002000200025
:104220002000200020002000560031002E00300029
:04423000300030002A
:00000001FF
